:0200000089284D
:080008000B1D0900A400030E0A
:100010008301A3000A08A5008A01061D1128A60174
:100020001628260FA6004620FF30B100061C1A280D
:10003000A7011F28270FA7004620FF30B100861D0B
:100040002328A8012628280FA80046202F083004BE
:1000500003192F28B00F2F28AF0F2F28B2152C0807
:10006000031DAC032D0A031938282D08031DAD0309
:10007000310803193E28B10B3E28321625088A00A4
:10008000230E8300A40824080B110900FC30AF00E4
:100090001830B00008008207543458340034523409
:1000A0005834003455344E3400344C344F344334D7
:1000B0004B3445344434003420342034003420346C
:1000C00044344934533450344C344134593420345A
:1000D00000344D3455344C34543400344D344134B0
:1000E000583400344D3449344E34203400342034F4
:1000F000563443344F3420344F344634463453342A
:10010000453454342034003420344D3448347A3467
:1001100000348316031360308F00831603130730F7
:100120009C00831603139B016A2321308400443012
:10013000A0008001840AA00B992803138316303095
:1001400085002D3086000430810083120617262298
:10015000861DB2168E238101A0308B004620B2117D
:10016000FB215830F2218430FC2109300222B219DF
:10017000AE28A2238030FC21861EC328321FB2176E
:1001800032175230C728321BB21732135430F221C3
:100190008230FC210630321DD028341FD028103088
:1001A0000222B21FD628B11BEE28B213321FE32859
:1001B0003930552372233D3063234E233F30632370
:1001C00041233930ED283B305523722343306323DC
:1001D0004E234530632341233B305C23DB219E21AA
:1001E000B72815242E1CB728F621133002221D3003
:1001F0000222B219AE28DB21E6232E18B80AF72313
:100200002E18B80301303802031808290130B8004D
:1002100015303802031C0E291430B800D7013808F5
:10022000D8000A305802031C1829D800D70A11290F
:100230008E30FC215708303EF2215808303EF22122
:10024000DD232E1CF928FB21263002220330022256
:10025000133002228B21B219AE28DB213D309321CD
:100260003D305C239E21DD232E1C2B29FB212230D7
:100270000222B219AE28DB213F30552372233D30D4
:1002800091213F305C239E21DD232E1C3929FB2147
:10029000033002222B300222B219AE28DB2141307A
:1002A000CA2141305C239E21DD232E1C4C29FB21D9
:1002B000263002220030022213300222B219AE2868
:1002C000DB214330932143305C239E21DD232E1C10
:1002D0005E29FB2122300222B219AE28DB214530F3
:1002E000552372234330912145305C239E21DD2329
:1002F0002E1C6C29FB21003002222B300222B21965
:10030000AE28DB214730CA2147305C239E21DD2304
:100310002E1C7F29AE28CA30FC2138300222F02161
:1003200008006323972955237223CE01CF014E2362
:100330005F30CE005030CF0041230800B2104C098E
:10034000C039031DAA29B214CC09CD090130CD074B
:100350000318CC0A3808CB000310CB0DCB0DCB070C
:100360004B08CB000310CB0DCB0DCB074B08CB00BC
:100370000310CB0DCB0DCB070A23B222C030FC21DA
:10038000563084000930A0000008F221840AA00B36
:10039000C429080055238030CC0672238130CE005A
:1003A0009030CF0041237E30CE007030CF004E23FE
:1003B0008030CC0608006022861EE429393055239F
:1003C00036305C234130E9293B30552336305C23FD
:1003D000473063232A233C22363055230800F1217D
:1003E000F1212030B600B70005170B2A0130FC219F
:1003F00018306B2308008130B600B70005130B22BC
:1004000005170800B5004B20FF3903190800F22139
:100410003508013E022A8B1386138316303085007F
:1004200083128517B70E0F30B7050508F03937046A
:100430008500851385170F30B6050508F039360499
:10044000850085134B30AE228B17080085013722BB
:10045000372237224230850085136A232830FC2159
:100460000830FC21F6210630FC210C30FC296A23DF
:100470004330850085130800B310321587230F30F1
:10048000CE00A030CF004E235D30CE00C030CF0074
:10049000412349306323382303195D2A49305C2303
:1004A0009322C23085224C0885224D088522AE3029
:1004B0008522FF30852298223413B31832110800A8
:1004C000341F662A2D08031D792A82229322C33005
:1004D00085220830A000AD220616AD22060C060CBF
:1004E000B40D0612A00B6B2AA9229F229822341B5E
:1004F0008222861E341F802A321D802A061308009D
:10050000061708006E30AD000800B5000830A000E6
:10051000B50D0318A922031CA4229F22A00B882A30
:10052000A9229F2208000616A922AD22A422A12AF0
:10053000A422AD220616AD22A922AD220800AD22CA
:100540000616AD2206120800861083168610831246
:10055000080083168614831208000F30A100A10B37
:10056000AF2A080003101830A000D701D901DC0120
:10057000DE01D40DD30DD20DDE0DDC0DD90DD70D5E
:10058000A00BE52A5E0EDD005C0EDA00590ED800E5
:10059000570ED60032105630FA225730FA22583011
:1005A000FA225930FA225A30FA2232145C30FA22F6
:1005B0002E30DB005D30FA225E30FA22B21C0800D9
:1005C000550884002D30800008005E30EE225C303B
:1005D000EE225930EE225730EE22B92A8400033041
:1005E0000007B500B519800030300007B500B51B15
:1005F0008000080084000F3000050319032B303EF3
:100600008000321408003218FF2A203080000408CD
:10061000D5000800D4014C08D2004D08D3000830A2
:10062000A000CB0C0318192BA00B112BD201D30166
:1006300008000310242BCB0C031C242B4D08D307DC
:100640004C0803184C0FD207D20CD30CD40CA00BBF
:100650001B2B08004F08CD074E0803184E0FCC0780
:1006600008004F08CD024E08031C4E0FCC020800B4
:100670004F084D02B5004E08031C4E0A4C023504CB
:1006800008004E08D0004F08D1000130CF070318F2
:10069000CE0A3823031C08005030522B382303188D
:1006A00008004E305523B314080084000008CC0025
:1006B000840A0008CD00080084004C088000840AE9
:1006C0004D088000080084000008CE00840A00085D
:1006D000CF0008007630A100A201A20B6D2BA10B68
:1006E0006D2B0800CE010130861D1430CF00EE23A3
:1006F0002E182A23FF232E1831230230861DC830DE
:10070000CF00E6232E182A23F7232E1831234C0975
:10071000C039031D0800CC01CD0108008312031766
:100720008D0138308312031384001130A000BD23E3
:100730008000831203178D0A83120313840AA00B0F
:10074000972B0800321E08003212831203178D0106
:1007500083120313383084001130A000BD2300023F
:100760000319B42B0008C623831203178D0A8312C2
:100770000313840AA00BAE2B0800831603170C1476
:10078000831203170C088312031308000C12831240
:1007900003178C00831603170C15831203138B1396
:1007A0008316031755308D00AA308D008C148312E8
:1007B00003138B170C1EDA2B08001E30B5002B0814
:1007C000AE00280208242808AB0008006430260286
:1007D000031CEE2B4630A6006630EF2B3C30B500F4
:1007E0002908AE00260208242608A9000800643063
:1007F0002702031CFF2B4630A7006630002C3C303C
:10080000B5002A08AE00270208242708AA0008001D
:100810000318122C2E08053C0318122C2E08350242
:10082000FF30031C0301AE000800DD232E1C08006E
:0E0830002C0803191C2C08001930AC00122CE7
:02400E00703F01
:02401000FC3F73
:1042000001004B0000004B0000004700E00054009C
:104210006000000000004700E00054006000000063
:0242200000009C
:00000001FF
